:020000040000FA
:040800008431492CCA
:100806000800843120007F08F1002100111E262CEB
:100816002000111E262C4E08A03E860087010108E6
:1008260023009A000130F00070082000CE071F3028
:10083600F0007008CE050130CD02CD08031D452C11
:1008460021001112452C2000911E412C230019086D
:10085600F00020004908203E86000130870070081D
:1008660081000130F0007008C9071F30F0007008E1
:10087600C9050130F0007008CA07452C0B1D452C30
:100886000B11FC1471082000FF00090084314B2C69
:10089600FC01FD01203084000030850030309731A6
:1008A600C1278431A0308400003085004230973162
:1008B600C1278431203084000130850020309731F3
:1008C600C12720008A31862A20003B1C782CFE3066
:1008D600E0006008BB053C08E0006008D800D901CC
:1008E600DA017B308B3170230800BB1C8B2CFD306A
:1008F600E0006008BB053C08E0006008D800043052
:10090600E1006108D900DA0104308B317023080058
:100916003B1E9E2CEF30E0006008BB053C08E00063
:100926006008D8000930E1006108D900DA01043016
:100936008B3170230800BB1D08004C08E000E10164
:10094600E009E109E00A0319E10A4E086007E2003E
:1009560061080318610AE30062081F3EE4000030E4
:10096600633DE5001F306405E60000306505E700DD
:100976006708803AFF0080307F02031DC42C0B30CD
:100986006602031C080001302000E0006008A8078A
:10099600F92D3C08E0006008D800D9012100420882
:1009A6002000E1006108DA007C308B3170230800FA
:1009B60020003C08E0006008D800D901D90A2100CF
:1009C60043082000E1006108DA007C308B31702397
:1009D600080020003C08E0006008D8000230E10072
:1009E6006108D900210044082000E2006208DA000C
:1009F6007C308B317023080020003C08E000600842
:100A0600D8000330E1006108D90021004508200024
:100A1600E2006208DA007C308B3170230800200087
:100A26003C08E0006008D8000430E1006108D90005
:100A3600210046082000E2006208DA007C308B3193
:100A46007023080020003C08E0006008D80005304C
:100A5600E1006108D900210047082000E200620891
:100A6600DA007C308B317023080020003C08E0005F
:100A76006008D8000630E1006108D9002100480866
:100A86002000E2006208DA007C308B317023080017
:100A960020003C08E0006008D8000730E10061084B
:100AA600D900210049082000E2006208DA007C3003
:100AB6008B317023080020003C08E0006008D80055
:100AC6000830E1006108D90021004A082000E20050
:100AD6006208DA007C308B317023080020003C0865
:100AE600E0006008D8000930E1006108D900210063
:100AF6004B082000E2006208DA007C308B3170235C
:100B0600080020003C08E0006008D8000A30E10038
:100B16006108D90021004C082000E2006208DA00D2
:100B26007C308B317023080020003C08E000600810
:100B3600D8000B30E1006108D90021004D082000E3
:100B4600E2006208DA007C308B3170230800200056
:100B56003C08E0006008D8000C30E1006108D900CC
:100B660021004E082000E2006208DA007C308B315A
:100B76007023080020003C08E0006008D80013300D
:100B8600E1006108D90021004F082000E200620858
:100B9600DA007C308B317023080020003C08E0002E
:100BA6006008D800F830E1006108D9003408E20096
:100BB6006208DA007C308B317023080020003C0884
:100BC600E0006008D800F930E1006108D90040086B
:100BD600E2006208DA007C308B31702308002000C6
:100BE600A801F730E0006008BB0508002808FF3EB2
:100BF600031CF22D8400103004020318F22D8831F4
:100C06000435283E82000800412F20003C08E00001
:100C16006008D8000430E1006108D9000A30E2001B
:100C26006208DA0005308B317023863120003C08DB
:100C3600E0006008D8000530E1006108D9000B30FB
:100C4600E2006208DA0005308B31702308002000CC
:100C56003C08E0006008D800D90121005D082000AA
:100C6600E1006108DA0005308B31702386312000FF
:100C76003C08E0006008D800D901D90A21005E08C6
:100C86002000E1006108DA0005308B3170238631DF
:100C960020003C08E0006008D8000230E10061084E
:100CA600D90021005F082000E2006208DA00053062
:100CB6008B317023863120003C08E0006008D800A4
:100CC6000330E1006108D900210060082000E2003D
:100CD6006208DA0005308B31702308002000C60850
:100CE600031D772E36160800EF30E0006008B605C3
:100CF6000800361E08008D3196250800361E0800AD
:100D0600BB150800361E08008A313D220800361E33
:100D16000800EF30E0006008B6050800361EA22E77
:100D26003C08E0006008D800D90121005D082000D9
:100D3600E1006108DA0005308B317023863120002E
:100D46003C08E0006008D800D901D90A21005E08F5
:100D56002000E1006108DA0005308B31702386310E
:100D660020003C08E0006008D8000230E10061087D
:100D7600D90021005F082000E2006208DA00053091
:100D86008B317023863120003C08E0006008D800D3
:100D96000330E1006108D900210060082000E2006C
:100DA6006208DA0005308B317023863120003C085A
:100DB600E0006008D8000430E1006108D9000A307C
:100DC600E2006208DA0005308B317023863120009C
:100DD6003C08E0006008D8000530E1006108D90051
:100DE6000B30E2006208DA0005308B317023863161
:100DF60020003C08E0006008D8000630E1006108E9
:100E0600D9000230E2006208DA0005308B31702327
:100E1600863120003C08E0006008D8000730E10079
:100E26006108D900DA01DA0A05308B31702308002F
:100E3600361E08003C08E0006008D8000830E100D3
:100E46006108D9008C319D2486312000E2006208B9
:100E5600DA0005308B3170230800361E080046087C
:100E6600E0006008C3000800361E0800B701B70A94
:100E760008000130E0006008C007080020004508AF
:100E8600013A0319712E033A03197C2E013A03190C
:100E9600812E073A0319852E013A03198A2E023A42
:100EA6000319912E0F3A03191B2F013A0319082E25
:100EB600033A03192A2EF03A0319302F043A03197C
:100EC600372F3C2F080020003508013A031D862FD6
:100ED6000130E3006308B1073108E4006408BC0090
:100EE6003C08E3006308D8004508E4006408D9001C
:100EF6004608E5006508DA0035088B31702387312E
:100F0600883182200800200031083C0603198E2F04
:100F16008A31CF22873120003108FF3A0319972FF3
:100F260031083C06031D080028302100C00023308C
:100F3600C100D92F20004508E3006308FD00080022
:100F460088318220080020003A080319AD2F873126
:100F5600F22708002000430803190800D801D90128
:100F66000230E3006308DA00FF308B317023200083
:100F7600080086310726200008008E311B26200037
:100F860008008931532120000800200045083C064E
:100F9600031908004608623A031D0800C201C20A86
:100FA60008000130E3006308C00708002000350888
:100FB600023A0319A32F013A0319A62F793A031906
:100FC600C82F073A0319C42F033A0319C02F013A51
:100FD6000319BC2FFF3A03199D2FD42F08002000B8
:100FE600BA01FD01BF0128302100C0002330C10035
:100FF600080020008E13CF0108008E311F2E8E317F
:10100600252E8E312C2E8E31332E8E313A2E8E3168
:10101600A12E8E31412E8E31482E8E314F2E8E319D
:10102600562E8E315D2E8E31642E8E316B2E8E3184
:10103600A12E8E31A12E8E31722E8E31792E8E31C9
:10104600802E8E31872E8E318E2E8431CC2C84319B
:10105600DB2C8431EC2C8431FF2C8531122D85312B
:10106600252D8531382D85314B2D85315E2D8531E8
:10107600712D8531842D8531972D8531AA2D8531A8
:10108600BD2D8531D02D8531E12D89315A29893102
:10109600572989316229893160298931672989313E
:1010A6006A298931702989317329F4008B13230049
:1010B60015137408920072089100151295161515ED
:1010C60073089300940195129731C72723001511D1
:1010D6008B17080023001D169D171E121D139E1642
:1010E6001E131E159F1522309B002000CC01CE0139
:1010F600CD01C901CB01CA012100911608002000CB
:101106004308031994283C08E0006008D80003301F
:10111600E1006108D900DA01FF308B317023883194
:1011260020002000B6018731FC272000BA01BA0A48
:1011360008002000CA08031DA228F93008004B0841
:10114600203E8600013087000108F2007208F30095
:101156000130F2007208CB071F30F2007208CB058F
:101166000130CA0273080800F601F701721CBF2895
:101176007408F6077508F73D0130F435F50D890B4F
:10118600C0280130F336F20C890BC52873087204A7
:10119600031DB9287708F301F3077608F201F20771
:1011A6000800F3007308F20020004C08A03E8600F9
:1011B6008701720881000130F2007208CC071F30E7
:1011C600F2007208CC050130F2007208CD0721004A
:1011D600111A080023009E1CED2821001116080094
:1011E6002000420803191429CA0803191B2988314B
:1011F6009C208831FB007B082000E90069088831C3
:10120600D42088312000E908031D12290130FB0093
:101216007B08AC07C8302C02031CF728C201AC01BE
:10122600F72805304A02031C1B298B31CE2388314F
:1012360023009D1C08001D121D1608002000D0006A
:1012460074182829D101D2012C298030D100003010
:10125600D200743651047306F5007508D700571886
:101266003729D301D4013B298030D3000030D40084
:10127600573653047206F5007508D70057184629E5
:10128600D501D6014A298030D5000030D600573620
:1012960055045006FF3AF5007508D70057080800B0
:1012A6002000361E080079292100C71708007F3064
:1012B600F20072082100C7050800B6160800DF30E4
:1012C600F2007208B6050800210047170800BF3073
:1012D600F20072082100C70508002100C7160800A1
:1012E600DF30F20072082100C7050800200045081B
:1012F6008400083004020318080088310435483E8B
:1013060082000800033020006102FC3003196002ED
:10131600031C9129FF30E20062089C296108E30062
:101326006008E200E336E20CE336E20C6208E40011
:101336006408FB000030FB08031D0130E200620870
:10134600CF008E177B08220099007B089B002000A7
:101356004308013A031D08003C08E2006208D80071
:101366000D30E3006308D9007B08E4006408DA0066
:10137600FF308B31702308008A313D2289310038D5
:10138600031D08006430F80078082100C200CD0172
:10139600CD0A4630F8007808CE003230F8007808DA
:1013A600CF008230F8007808C3003230F8007808A1
:1013B600C4000A30F8007808C5007D30F8007808C7
:1013C600C6000430F8007808C8002030F800780815
:1013D600C9004030F8007808CA00FF30F8007808E5
:1013E600CB00A030F8007808C7008D31962508009C
:1013F600FB0079082000D000D1015008A000510858
:10140600A1007B08D000D101D009D109D00A031967
:10141600D10A78085007F20051080318510AF30060
:101426002108F501F5072008F401F4078831B720F3
:10143600893173082000A101A1077208A001A00745
:101446007A08FE3E890A292AA136A00C890B272A8A
:101456007B08D000D101D035D10DD035D10D500843
:10146600A0075108A13D2108F901F9072008F80154
:10147600F80708002000C808031D842AC230F600B9
:101486007608D0005530F6007608D1002030F600F8
:101496007608D400203054020318552A2030F6006E
:1014A6007608D400D3015408530203187A2A530845
:1014B600F6007608F2003F309731EF278A31F700C1
:1014C60077082000D2005208F6007608D1075208A5
:1014D600F600500886008701760881000130F60084
:1014E6007608D0070130F6007608D307562A510849
:1014F600003A003003190130F6007608C8004808A3
:101506000800013008002000EE018D3118258A31CF
:10151600200037080319932A00308A000828200083
:101526008831F3208A31FC1CC42AFC1001302000CB
:10153600ED006D08BD07BA08031DBB2A2100C71FB1
:10154600BB2A0130C0020030C13B41084004031DE4
:10155600BB2A20003C08ED006D08D800D901D90A45
:10156600DA01FF308B3170238A31883182208A314B
:1015760064002000BA08031DC42A0230ED006D087D
:101586008E062000BA08031DCB2A8F3151278A31D7
:10159600843167248A318B2A2100111220003508F4
:1015A600F2004C08A03E86008701720881003108CF
:1015B600F2000130F3007308CC074C081F39A03E37
:1015C60086008701720881004508F2000130F300A9
:1015D6007308CC074C081F39A03E860087017208A5
:1015E60081004608F2000130F3007308CC074C086E
:1015F6001F39A03E86008701720881003308F20079
:101606000130F3007308CC074C081F39A03E860052
:101616008701720881000130F2007208CC071F3082
:10162600F2007208CC050530F2007208CD072100E1
:1016360011160800F801F31F272BF209F309F20A25
:101646000319F30AF801F80AF51F322BF409F50914
:10165600F40A0319F50A0130F6007608F806F901CE
:10166600FA01730872040319612BF701F70AF31BD9
:10167600462B0130F235F30D890B3D2B0130F60078
:101686007608F7073A2B0130F935FA0D890B472B07
:1016960073087502031D512B72087402031C582B24
:1016A6007208F4027308F53B79140130F336F20C34
:1016B600890B592B0130F702031D462B78080319B5
:1016C600692BF909FA09F90A0319FA0A7A08F301E2
:1016D600F3077908F201F2070800FA002100111257
:1016E6007A082000DB004C08A03E860087015B08D4
:1016F60081005808DB000130DC005C08CC074C0890
:101706001F39A03E860087015B0881005908DB006F
:101716000130DC005C08CC074C081F39A03E86006F
:1017260087015B0881005A08DB000130DC005C0899
:10173600CC074C081F39A03E860087015B08810054
:101746005808DB005B08F2005908DC005C08F3006F
:101756005A08DD005D08F4007A088931212120004D
:10176600DE000130DF005F08CC074C081F39A03EC1
:10177600860087015E0881000130DB005B08CC072C
:101786001F30DB005B08CC050530DB005B08CD07AE
:1017960021001116080020004B08203E860001306B
:1017A60087000108E6006608B5004B08013E1F39B0
:1017B600203E8600013087000108E6006608B10079
:1017C6004B08023E1F39203E860001308700010883
:1017D600E6006608C5004B08033E1F39203E86001A
:1017E600013087000108E6006608C6004B08043E83
:1017F6001F39203E8600013087000108E600660892
:10180600B3003108E6006608F2004508E7006708FD
:10181600F3004608E8006808F400350889312121FC
:101826008B3120003306031D232C4B08053E1F3940
:10183600E6006608CB000530CA0287316627080035
:1018460001302000E6006608B4074B08013E1F3948
:10185600E6006608CB000130CA0208002000E90154
:101866002100C71E472C20006508E6006608D20046
:1018760069088E31A2268C3120005308A501A507E0
:101886005208A401A407542C20006508E600E701CD
:101896006608A4006708A5000230A435A50D890BCB
:1018A600502C6908E600E701E635E70DE635E70D59
:1018B6006608A4076708A53D03302502ED30031925
:1018C6002402031C6A2CEC30A4000330A500430854
:1018D600013A031D7E2C3C08E6006608D8000A3053
:1018E600E7006708D9006908E8006808DA00FF30F1
:1018F6008B3170238C3120004308013A031D932C51
:101906003C08E6006608D8000B30E7006708D900F7
:101916006508E8006808DA00FF308B3170238C31E7
:1019260020002508E101E1072408E001E0078931EC
:101936008521080021001D08F80078082000A9006C
:1019460021001E08F80078082000AA002200971639
:10195600171621001D08833974389D001D149E1723
:101966001E088F3920389E00FC309E051E118330DC
:10197600F800F80BBC2C21009D149D18C02C1C08E7
:10198600F800F90178082000A2007908A3002208CF
:10199600F900F8017808A2007908A30021001B08C5
:1019A600F800F90178082000A2047908A3043B3066
:1019B600F2000030F3002308F501F5072208F401D0
:1019C600F4078831B7208C3173082000A301A307E0
:1019D6007208A201A2072308F9002208F8000630BF
:1019E600F936F80C890BF32C7808A2007908A300C5
:1019F60021004608383EF800013003180230F9008D
:101A060078082000A2027908A33B2208F80078088B
:101A1600C400290821009D0020002A0821009E00FC
:101A2600220097122000440808007830210099040B
:101A36000730980091012000910112303C00A4006B
:101A460014303D00A30025009A0120008E018D016F
:101A56008C01FF3021008C00FF308D00FF308E009E
:101A6600FF3023008C00FF308D008E0121000E1008
:101A76008E108E110E128E1323000E1721001D14C8
:101A86001D08833948389D009E131E088F3920385B
:101A96009E00FC309E051E11073022009100640056
:101AA6002100951195121508F83902389500200085
:101AB600950121001708C1391638970017146400DC
:101AC6002000B401C001C301C201B70188316D20F5
:101AD6008D318931BF218D319731D0278D318431B8
:101AE60003248D312000B801B601B501B001A6016D
:101AF600A701210042082000EA006A08BE00E501AD
:101B060000308C3131248D310A302000EA006A0819
:101B1600B2006530EA006A08BC00BB018831822049
:101B2600E0308B000800C230F60076082000D300B3
:101B36002030F6007608D400203054020318A72D72
:101B46002030F6007608D400D101D10AD501540818
:101B560055020318CA2D5508F6007608F2003F30E4
:101B66009731EF278D31F70077082000D000530812
:101B76008600870101085006031DD1010130F600D9
:101B86007608D3070130F6007608D507AA2DD108C6
:101B9600031D08005530F6007608D200C230F60064
:101BA6007608D3002100E1012000D5015408550232
:101BB6000318ED2D5308860087010108F600760804
:101BC600D2070130F6007608D3070130F600760812
:101BD600D507D92D5203FF3AF60076082100E10019
:101BE600F2013F309731DF278D31C230F60076089B
:101BF6002000D300D50154085502031808005508E3
:101C0600F6007608F2005308860087010108F700FF
:101C16007708F3003F30883158208D310130F600C7
:101C260076082000D3070130F6007608D507FE2D8A
:101C36002000361E0800952E4608F2007208210084
:101C4600C200080020004608F20072082100C30006
:101C5600080020004608F20072082100C4000800AF
:101C660020004608F20072082100C5000800200086
:101C76004608F20072082100C60008002000460847
:101C8600F20072082100C800080020004608F20091
:101C960072082100C900080020004608F2007208F8
:101CA6002100CA00080020004608F2007208210040
:101CB600CB00080020004608F20072082100CC0084
:101CC600080020004608F20072082100CD00080036
:101CD60020004608F20072082100CE00080020000D
:101CE6004608F20072082100DD00080020004608C0
:101CF600F20072082100DE00080020004608F2000B
:101D060072082100DF00080020004608F200720871
:101D16002100E000080020004608F20072082100B9
:101D2600CF00080020004508840014300402031880
:101D3600080088310435003E8200080008002000B3
:101D4600D900413052020318C12E21004808200054
:101D5600D4005408F8005208D5005508F90006309A
:101D6600D6005608FA0000308931FB217908200098
:101D7600D301D3077808D201D20708008130520276
:101D86000318E02E210049082000D4005408F8006A
:101D96005208C03ED5005508F9000630D600560850
:101DA600FA00210048088931FB2179082000D30177
:101DB600D3077808D201D2070800C13052020318AF
:101DC600FF2E21004A082000D4005408F8005208CB
:101DD600803ED5005508F9000630D6005608FA00B0
:101DE600210049088931FB2179082000D301D30756
:101DF6007808D201D20708005908D400D501D409C1
:101E0600D509D40A0319D50A5408FB3ED60000307A
:101E1600553DD7005708803AD80080305802031D38
:101E2600182F21004B08200056020318362F2000D9
:101E36005903FF3AFB3ED4005408F8005208403ECE
:101E4600D5005508F9000630D6005608FA002100DC
:101E56004A088931FB2179082000D301D307780885
:101E6600D201D207080021004B082000D4005408F4
:101E7600F8005208403ED5005508F9000630D60055
:101E86005608FA0021004A088931FB21790820000A
:101E9600D301D3077808D201D20708007C1C672F2C
:101EA60020002F083D0203185D2F7D08EA006A080E
:101EB600BF0008007D08EA006A08E5002100420824
:101EC6008C3131248F317C107D082000EA006A08AD
:101ED600BF007D08EA006A08E500210042088C314F
:101EE60031248F317D0803197B2F2000C1010800A2
:101EF6002000B00803190800AD08031D882F30081C
:101F0600EA006A08AD0030089A2F0230F20000306D
:101F1600F3002D083007F400F501F50D8B311D2374
:101F26008F3172082000EA006A08AD002D08EA0029
:101F36006A08AE00B0010C3041020318A72F013029
:101F4600EA006A08C107080021004408013E200093
:101F5600EA00003003180130EB006B08803AEC0011
:101F660080306C02031DB92F2E086A020318EB2F6E
:101F760001302000EA006A08B2073208143A031D4D
:101F86000800193021004202031CE12F0130C20271
:101F96004408143E2000EA00003003180130EB002C
:101FA6006B08803AEC0080306C02031DDC2F2E0893
:101FB6006A020318E12F01302100C2020A30200014
:101FC600EA006A08B2000A30EA006A08AF00672F22
:101FD6002100440820002E02031808000130B20236
:101FE600031D08000130EA006A082100C2070A3012
:0A1FF6002000EA006A08B2000800AB
:102F8200640080010131890BC22F003455302300C7
:102F92009600AA3096009514000000000800A030A8
:102FA20022009800990123000C158C150C16A030F4
:102FB20022009A009B0123008C160800F3008B1359
:102FC2002300151373089200720891001516151547
:102FD2009731C727230015118B170800F40023002F
:102FE2001513740892007208910015140000000075
:0E2FF20023001308F3007308F50075080800AB
:00000001FF
